:020000040000FA
:020000003528A1
:08000800A800A60F2228A70A98
:100010002708223C031D222886110611061386128A
:1000200006120B3026208700861778228613762248
:100030000130A51C023026208700861778228613FF
:1000400076221128A0308B002808090082073F344F
:1000500006345B344F3466346D347D3407347F347A
:100060006F344034793471347334850186018701EB
:10007000A501831606309F003F3085008601870169
:1000800020308B00D730810083120A302620870071
:100090000A30A2008717762287137622851C5528FE
:1000A000051C5528A20B4A285F280D302620870002
:1000B000251466227622051C5A28851C5A288B177F
:1000C000A510A601A701051A74280B302620870069
:1000D000662276226622762266220615051E6E2884
:1000E0004B224B2206118B130130262087006622FB
:1000F0007622051C7828051C8028851C17297B285A
:1001000002302620870066227622051C8428051CE2
:100110008C28851C1D29872803302620870066220D
:100120007622051C9028051C9828851C2A299328CE
:1001300004302620870066227622051C9C28051C98
:10014000A428851C37299F28053026208700662291
:100150007622051CA828051CB028851C4429AB283C
:1001600006302620870066227622051CB428051C4E
:10017000BC28851C5129B728013026208700871705
:1001800066227622051CC128051CC928851C672902
:10019000C428023026208700871766227622051C95
:1001A000CE28051CD628851C6D29D1280330262091
:1001B0008700871766227622051CDB28051CE328AA
:1001C000851C7B29DE2804302620870087176622BD
:1001D0007622051CE828051CF028851C8929EB28B7
:1001E000053026208700871766227622051CF52811
:1001F000051CFD28851C9729F82806302620870035
:10020000871766227622051C0229051C0A29851CEF
:10021000A529052907302620870087176622762220
:10022000051C0F29051C7428851CB3291229662278
:10023000CA21F221063002220E2266220230262036
:100240008700251C252985181D29D421F221063077
:1002500002220E226622033026208700251C322926
:1002600085182A29D421F221063002220E22662284
:10027000043026208700251C3F2985183729D421E2
:10028000F221333002220E2266220530262087001A
:10029000251C4C2985184429DE21F2211830022220
:1002A0000E226622063026208700251C5929851833
:1002B00051291A220C3026208700532205185E2966
:1002C0000A30262087007622051C632974286622BE
:1002D000CA21F221063002220E2266220230262096
:1002E00087008717251C762985186D29CA21F221D8
:1002F000153002220E22662203302620870087173F
:10030000251C842985187B29D421F221153002224D
:100310000E2266220430262087008717251C92298A
:1003200085188929D421F221333002220E22662237
:100330000530262087008717251CA02985189729B6
:10034000D421F221153002220E2266220630262008
:1003500087008717251CAE298518A529DE21F221E3
:100360005A3002220E226622073026208700871785
:10037000251CBC298518B3291A220C302620870099
:1003800053220518C1290A30262087007622051C31
:10039000C629BC282830A200861464306B2286103F
:1003A0007822A20BCC2908002830A20086147830CD
:1003B0006B2286107822A20BD62908002830A200D2
:1003C0008614C8306B2286107822A20BE029080020
:1003D0002830A20086149B306B2286107822A20B54
:1003E000EA2908008B17A514A601A701861505198F
:1003F000FC29851EFF29F629051EFF29F6298611ED
:100400008B130800A30086160708A4003822861262
:10041000240887004B22A30B032A08008B17A51082
:10042000A601A7010615051E132A4B224B22061111
:100430008B13080085190800051A242A0615051EC5
:100440001F2A4B224B220611061706154B224B2260
:100450004B224B224B224B220430A30006154B2289
:1004600006114B224B224B22A30B2E2A0613080007
:100470000A30A2003E22A20B3A2A08002030870050
:1004800076220130870076220230870076224030C3
:1004900087007622080028304E2A0430A2007622F7
:1004A000A20B4F2A08008617762276228613762220
:1004B0007622861776227622861376227622861771
:1004C00076227622861376227622080086177822F4
:1004D000861378220800A000000000000000000041
:1004E000000000000000A00B6C2A0800FA30792AF6
:1004F0003230A1006E30A0000000000000000000BB
:0E05000000000000A00B7C2AA10B7A2A080044
:00000001FF
